:1000000009C02EC015C049C013C012C011C010C015
:100010000FC00EC011241FBECFE9CDBF20E0A0E667
:10002000B0E001C01D92A236B207E1F77BD075C1E6
:10003000E7CF399A3D9A86B1876886B90895369A8E
:100040003699FECF85B190E0089585B7836085BF6E
:100050008BB780648BBF89B7826089BF789408951D
:100060001F920F920FB60F9211248F939F9312BE7F
:100070001FBC83B7836083BFB19B08C082B790E089
:100080009093610080936000B199F8CF9F918F9118
:100090000F900FBE0F901F9018951F920F920FB6E2
:1000A0000F9211248F939F93809160009091610033
:1000B000019690936100809360009F918F910F90C3
:1000C0000FBE0F901F901895C09A87EC9FEA01977A
:1000D000F1F700C00000C09887EC9FEA0197F1F7A4
:1000E00000C00000C09A87EC9FEA0197F1F700C0BA
:1000F0000000C09887EC9FEA0197F1F700C000006C
:10010000C09A87EC9FEA0197F1F700C00000C09801
:100110009FE329E181E0915020408040E1F700C059
:1001200000000895B89AB99884DF8FDF88DF9C01BA
:100130002B5531092C323105C0F0225331092C32B4
:100140003105A8F0225331092733310590F0C297C9
:1001500094F4C09A2FE78CEF9AE0215080409040B1
:10016000E1F700C00000C0E007C0C2E005C0C3E086
:1001700003C0C4E001C0C9E062DF2091600030919B
:1001800061002D5031092231310508F482C0C09A36
:100190008FEB9DE50197F1F700C00000C0988FEB51
:1001A0009DE50197F1F700C00000C09A8FEB9DE537
:1001B0000197F1F700C00000C0988FEB9DE5019713
:1001C000F1F700C00000C09A8FEB9DE50197F1F7B1
:1001D00000C00000C0988FE295E70197F1F700C0DA
:1001E0000000C09A87EC9FEA0197F1F700C0000079
:1001F000C09887EC9FEA0197F1F700C00000C09A11
:1002000087EC9FEA0197F1F700C00000C09887ECE7
:100210009FEA0197F1F700C00000C09A87EC9FEABF
:100220000197F1F700C00000C09887EC9FEA0197A2
:10023000F1F700C00000C09A8FEB9DE50197F1F740
:1002400000C00000C0988FEB9DE50197F1F700C05A
:100250000000C09A8FEB9DE50197F1F700C0000008
:10026000C0988FEB9DE50197F1F700C00000C09AA0
:100270008FEB9DE50197F1F700C00000C0989FEB60
:1002800024ED81E0915020408040E1F700C0000063
:1002900073CF8036910524F4C23011F415DF6CCF92
:1002A0008139910524F4C33011F40EDF65CF813C10
:1002B000910524F4C43011F407DF5ECFC93059F53D
:1002C000C09A87EC9FEA0197F1F700C00000C09840
:1002D00087EC9FEA0197F1F700C00000C09A87EC15
:1002E0009FEA0197F1F700C00000C09887EC9FEAF1
:1002F0000197F1F700C00000C09A87EC9FEA0197D0
:10030000F1F700C00000C09887EC9FEA0197F1F771
:0E03100000C0000031CFC0982FCFF894FFCF6F
:00000001FF
